:020000020000FC
:1000000017C016C015C014C013C012C011C010C054
:100010000FC00EC00DC04C474D303331323237491E
:10002000203130306D730A0D0000204B487A0000FB
:100030005FED5DBF59E159B95FEF52BB50E451BB71
:10004000A3D038D0A1D00BD057D0FECF51E0252E71
:1000500051E0352E54EF452E57E2552E089551E0CC
:10006000252E5AE0352E54EF452E57E2552E089591
:1000700051E0252E54E6352E54EF452E57E2552EED
:100080000895539A5D9BFDCFACB953980895F0E065
:10009000E6E201D00895C895002021F0A02DF1DFFF
:1000A0003196F9CF0895F7DFF2DF0895F0E0EAE244
:1000B000F2DF0895F0E0E6E1F6DF08954B2F469574
:1000C000469546954695405D4A3308F0495FBF70B6
:1000D000B05DBA3308F0B95F0895F0DFA42FD1DF27
:1000E000AB2FCFDF089558E0A0E3BB1F08F4A1E3D6
:1000F000C8DF5A95C9F7089550E95AB9789450E085
:100100005FBD50E05DBD5CBD56E05EBD122C9698B3
:10011000832D642D752D6A956030E9F77A957030DE
:10012000D1F7000000008A95A1F71A9489F750E0F2
:100130005EBDF894969A0CB51DB50DD0A8DFAF2D15
:1001400050E3A50F9EDFBE2DC8DFAEE29ADFBD2DC6
:10015000C4DFACDF089520E1FF24EE24DD24FF2777
:10016000000F111FDD1CEE1CFF1C2A9509F40895D9
:10017000E0E132913D5F33FD30833081305D37FD0A
:100180003083ED30B1F7ECCF73DF122C832D642D6B
:10019000752D6A956030E9F77A957030D1F78A95B8
:0801A000B1F71A9499F70895D4
:00000001FF
